:020000040000FA
:020000000000FE
:100200001E290408FA008C1E1429261A0929691AC5
:1002100087168313680869071F39C03E84001A08CF
:100220008000E90AE91AE9037D088A007A08840057
:100230007C088300FB0E7B0E8B1709008A150A12BF
:10024000FF248A150A12782601308A00861B2B2982
:100250008A150A1215268A150A120E268A150A12FE
:1002600046258A150A12F1250830F3008A110A1270
:10027000E4218A150A12B225022701308A0083126E
:100280000313261E48298316981C482983128712B7
:100290008312A41C702918191A08981C51291812C5
:1002A0001816E908031D5729261E87126B29831685
:1002B0008C12831283136808C03E84000008B000CB
:1002C000E903E80A1F30E80583168C16831230080C
:1002D0008A110A12162201308A00EB08031D6F26CC
:1002E0000B19752101308A003F29383081000B112C
:1002F0009B0B95290A309B00D708031DD70B822939
:100300003708B6009C0B95290A309C00241C9529BF
:100310005A25031D8D2926139529261B9529A830BA
:10032000ED266A250130B600261783120313B408A0
:100330000319A52983160313A01783120313B4030B
:10034000B408831603130319A01383120313E421C3
:1003500083120313A61DB92983132108B03E84001C
:1003600000087F39B10035020319B9293108B600F8
:10037000B50001308A00360A0319C1298A150A120C
:10038000ED23A41E08008A150A12722401308A0087
:10039000A71DCF298A150A122A2401308A006E1F50
:1003A000080083120313ED1BDD29271808006E13C4
:1003B0006D08E0000130EB006F2E6E136D08B60083
:1003C0008A150A12ED230800831203137308B10083
:1003D000831331089F3E840000080925B0003108CE
:1003E0007302A83E84000008093A0319F829FC2981
:1003F000300EFF3A0F39B000083084073008800013
:10040000B10BE92985168512080000308008031910
:100410000C2A643E800B092A840A80080319132AD7
:100420000A3E800B102A840A000708008312031377
:10043000B00002308A00831203133F088207362A75
:10044000442AAD2A042B6A2B942BF72B112CAA2BB0
:10045000C52B402C982C5A2B632BC22CF42AC22C6F
:10046000832B412BC22C1C2C232C292C1B3030021B
:10047000031D412A0130A6180C30BF000330C20012
:100480000800A61CC22C08004C303002031D4B2A69
:100490000230BF0008004B303002031D522A0330E7
:1004A000BF00080054303002031D592A0430BF0039
:1004B000080053303002031D602A0530BF000800D9
:1004C00050303002031D692A0330C1001830C000CB
:1004D0003B2C43303002031D702A0730BF00080058
:1004E00046303002031D772A0830BF0008003F3035
:1004F0003002031D7E2A0930BF000800453030025B
:10050000031D872A0330C1002730C0003B2C653013
:100510003002031D902A0930C1004830C0003B2C36
:1005200026303002031D972A0630BF0008005B30DA
:100530003002031D9E2A0730BF00080044303002FD
:10054000031DA42A2610AE2B41303002031DBB2C04
:100550000230C1004530C0003B2C4B303002031D3F
:10056000B82A0130C1000A30BF000330C0000800C3
:1005700041303002031DC12A0230C1003030C000BA
:100580003B2C43303002031DCA2A0330C100003027
:10059000C0003B2C4C303002031DD22ABF01083072
:1005A0008A00E7286C303002031DDA2ABF010930C7
:1005B0008A0041293F303002031DE12A0F30BF007D
:1005C00008005A303002031DEA2A0A30C1002130E7
:1005D000C0003B2C42303002031DBB2C0130C10057
:1005E0003330C0003B2C080041303002031DFC2A90
:1005F000BF0108308A00D12843303002031DBB2CD4
:10060000BF0108308A00FE284D303002031D0F2B39
:100610000130C1000A30BF001530C00008003F3073
:100620003002031D162B1230BF0008005330300279
:10063000031D1E2BBF0109308A00DA295230300217
:10064000031D262BBF010A308A000C2A72303002AB
:10065000031D2E2BBF018A110A12002841303002DF
:10066000031D372B0130C1001E30C0003B2C7330FE
:100670003002031D402B0730C1004230C0003B2C2C
:10068000BB2C4D303002031D492BBF010A308A00BC
:10069000312A50303002031D522B0130C1003C3052
:1006A000C0003B2C45303002031DBB2CBF010A307B
:1006B0008A006C2A4B303002031D612B0D30BF00C5
:1006C0000800BF01080041303002031D682B322BA7
:1006D000BF0108004B303002031D732B0530C100F1
:1006E0000630C0003B2C43303002031D7C2B03300E
:1006F000C1000930C0003B2C3F303002031DBB2C31
:100700001130BF0008004B303002031D8B2BBF019E
:100710000A308A00CC2A43303002031DBB2C013042
:10072000C1002D30C0003B2C47303002031D9F2BF1
:100730000130C1000A30BF000C30C0000800453055
:100740003002031DBB2C0130C1000A30BF0036301F
:10075000C00008005A303002031DB32B0130C10025
:100760002A30C0003B2C50303002031DBC2B01301E
:10077000C1003930C0003B2C54303002031DBB2C6B
:100780000230C1003F30C0003B2C54303002031D0A
:10079000CD2BBF0109308A00BD2956303002031D20
:1007A000D52BBF0108308A003D2841303002031D9F
:1007B000DD2BBF0108308A00772850303002031D3E
:1007C000E62B0130C1001B30C0003B2C453030020D
:1007D000031DEF2B0230C1002430C0003B2C4930F8
:1007E0003002031DBB2CBF0108308A00A82823302B
:1007F0003002031DFF2BBF0108308A00E728433079
:100800003002031D082CBF0107308A000F304C2F27
:1008100044303002031DBB2CBF0107308A000C306E
:100820004C2F4B3030020319D62A03303005BC0060
:10083000BC0A1430BF0008003B303002031DBB2C43
:100840001530BF00080030080F39BD001630BF005A
:10085000080048303002031D322CBF01BD0A8A1146
:100860000A12712F30080F390A3EBD0B342CBD001F
:100870001630BF0008000A3026180B30BF000800F1
:1008800041088313473E840030088000C10B0800F4
:10089000BF0104308A00400882078A150A12142911
:1008A0008A150A1252298A150A12CD298A150A12A6
:1008B000E82A8A150A126C2B8A110A12BB2C8A119B
:1008C0000A12BB2C8A150A12152A8A150A123A2B0B
:1008D0008A150A124F2B8A150A12BC2A8A150A1287
:1008E00098298A150A12842B8A150A12AA2B8A15AE
:1008F0000A12E42B8A150A12FC2A8A150A12832985
:100900008A150A1278298A150A12792B8A150A1271
:100910001D2C8A150A12542A8A150A12212C8A15AE
:100920000A12F0298A150A1295288A150A12BA2B7A
:100930002C303002031DA02CCC24C10B0800482C05
:100940003B303002031DB12CCC24C1030319482CC9
:1009500083134108473E840080018403C10BAC2C03
:10096000482C42080319C62C483C840030080F3933
:100970008000C2030800BF010330C20000308A11AA
:100980000A12742E30088A110A12F42EBF010330A5
:10099000C2008A150A12262C453084000008B100D6
:1009A000C2080319D62C8403C20BD32C0522B10034
:1009B0004108473E840031088000C301C401C501DD
:1009C000C601C7010330C200080083120313EB08FD
:1009D000031908000C1EEA2CEA018313603084001E
:1009E000261EF52C87165430ED2600089900EA0AD9
:1009F0006B086A020319002D840A0C1EFD2CF52CCD
:100A0000EB010800831203131F151F19052D1E0883
:100A1000080083120313B3000830B200031005115D
:100A20008510B31B851485190314B30D051500003B
:100A3000B20B0E2D0511330808000830B200083043
:100A4000ED260711831607110830ED2683160715CA
:100A5000831203130830ED260314071D0310B10C95
:100A60006430ED26B20B1F2D3108080083120313EA
:100A7000B1000830B200831203130830ED260711CD
:100A80008316031307110830ED2683120313311C5C
:100A90004C2D831603130715831203136430ED26C0
:100AA000831603130715831203130310B10CB20B43
:100AB0003D2D0800831203130711831607118312BB
:100AC000E1268316071583126430ED260315071DF2
:100AD000031108003330362500000830B0008313BE
:100AE000B83084001D258000840AB00B722D83125B
:100AF0000800831203178D00831603178C130C1440
:100B00000C18802D83120C0803130800831203179E
:100B10008C00831203133908831203178D00831688
:100B200003178C130C15831203130B08B2008B13DD
:100B30008316031755308D00AA308D008C148C1845
:100B40009F2D8312031332088B00831203170C08A6
:100B50008312031308001030A61A103EA6133A029F
:100B60000318A6178316031391144426A03083128A
:100B70000313A61B023E4026442683160313111BB3
:100B80003A2E83120313A61FCA2D1030A61A103E48
:100B90003A02CB2D3A080000402644268316031360
:100BA000111B3A2E831203133B084026442683165A
:100BB0000313111B3A2E8316031391144426A130FC
:100BC00083120313A61B023E4026442683160313FA
:100BD000111B3A2E911544268316031391161116F4
:100BE00011154426831203131308080083120313FC
:100BF000B2001030A61A103EA6133A020318A61728
:100C00008316031391144426A03083120313A61BEA
:100C1000023E4026442683160313111B3A2E8312EC
:100C20000313A61F182E1030A61A103E3A02192ED2
:100C30003A084026442683160313111B3A2E8312CA
:100C400003133B084026442683160313111B3A2E38
:100C50008312031332084026442683160313111B04
:100C60003A2E83160313111544268A110A12EA2616
:100C700006300800831603131115442615300800AA
:100C8000831203139300003483120313FA30B3006A
:100C9000B30B4D2E3E2E583008008C1D482E8C1163
:100CA00000348316031391144426E0304026442672
:100CB0006B0840264426EA01831360308400000854
:100CC00040264426EA0A6B086A020319692E840A40
:100CD0005F2EEB01831603131115442608008312BF
:100CE0000313A518E52C0800B10006308A0031086E
:100CF0008626B1009326FF39031908008A110A12CB
:100D0000F42606308A003108013E792E820700342D
:100D100005340D3414341B34203425342A34303453
:100D200036343C344434820743344D3444343F3405
:100D30000034433454342034563432342E3439346D
:100D40000034523453343234333432342C3400349B
:100D5000523453343434323432342C3400344C343E
:100D6000433444343A3400345034613472343F34C0
:100D7000003439343634303430340034313439349A
:100D80003234303430340034333438343434303462
:100D90003034003435343734363430343034003481
:100DA00049346E34693474342E342E342E34003485
:100DB0002C344134643472343A340034C830B200D4
:100DC000E32E0630B2000030B300B30BE52EB20BB9
:100DD000E32E08002230B200E32E83120313B30087
:100DE0000000B30BF02E0800B0000D303002031DE0
:100DF000FC2E0130BD00002F0A303002031D062FEB
:100E00003C0822020319BC01BC0A712F07303002D2
:100E1000031D0F2F831203130530B400080009309F
:100E20003002031D192F3D08F839073EBD003D274C
:100E3000712F20303002031C08000830B3008313E8
:100E4000E73084003008000203192A2F8403B30B13
:100E5000222F2D2FB3033308B0002F273D2F323020
:100E6000ED2630088800891009153E1A86163E1EA8
:100E700009140000091086120800BD0A3D0823026B
:100E8000031808000130BD00BC0A3C082202031808
:100E9000712F0130BC00712FB2003230ED263208C4
:100EA0008800891009113E1A86163E1E091400009A
:100EB000000009108612080083160313FF30880013
:100EC0008312091189140914000000000910080890
:100ED000B200B21B5C2F8910831600308800831289
:100EE0000800A2187C2F3E1E7C2F0C304C273E128F
:100EF00003303E050C3E4C273C08023C031C822F6D
:100F000000309C2F2308103C031C882F10309C2F8E
:100F10002308143C031C8E2F14309C2FA21C922FEC
:100F200028309C2F3E1A7C2F0C304C273E16033065
:100F30003E050C3E4C2700303C1C403E3D07031054
:100F4000FF3E80384C2FB1000330EB00800164304D
:100F5000B102031CAD2F800AA82FB1080319B22FCC
:100F60006430B10780080319B92F30308007840A34
:100F7000BA2FEB0380010A30B102031CC12F800A93
:100F8000BC2FB1080319C62F0A30B1076B18CD2F3B
:100F90008008031DCD2FEB03D02F30308007840A4B
:080FA0003108303E800008001A
:10100000831203138313261818284108EB00473076
:101010008400410884070008B1005F308400410863
:10102000840731088000C10B07288A110A126F2E2D
:1010300047308400410884070008B1006030840014
:1010400031088A110A12A3278A110A126F26083062
:101050008A00C10B2C2836282C30E0000130EB0030
:101060008A110A126F268A150A1218283B30E000EE
:101070000130EB008A110A126F2E831203135630CF
:10108000E0003A30E100261850283230E2002E30DD
:10109000E3003930E4000530EB008A110A126F2EAC
:1010A0003230E2002E30E3003930E4002C30E5002D
:1010B0000630EB008A110A126F26B10183136030EB
:1010C00084000130B9000630B10039088A110A12D3
:1010D00079258000B90A840A08308A00B10B652896
:1010E0003B3080000730EB008A110A126F2E8A1104
:1010F0000A12022508308A00831203134130E000EF
:101100003A30E1000230EB008A110A126F261E0805
:10111000C900031083161E0D8312C800C80DC80D28
:101120000230C1008A150A12002848080319A528B0
:10113000480B9C289701080083168710FF30920007
:101140008312043092003C30970049089500080053
:10115000831203134930E0003A30E1000230EB0023
:101160008A110A126F2608308A000830B100483010
:10117000B3008313B730310784000008B000831335
:1011800033088400B30A30088000B10BB9288316F5
:101190000313B801831203130830C1008A150A1221
:1011A0000028831203134C30E0004130E1003A3054
:1011B000E2000330EB008A110A126F262208C900F0
:1011C0002308C8000230C1008A150A120028013025
:1011D000B0003E128A110A124C273E1630084C27E6
:1011E0008A110A12E126E126013083120313BC00A2
:1011F000BD003E1208008A110A12712F83120313D8
:101200004C30E0004330E1003A30E2000330EB00C4
:101210008A110A126F263C08C9003D08C800023036
:10122000C1008A150A1200280C308A0029304902B0
:101230000318262C4908031DBD0000308A00243005
:1012400083120313FF0097301428A2034A08BD003D
:10125000831605304A020318262C4A08031DBC00D9
:10126000C80803193E29C81CC801FC30BE0503305C
:101270004805BE070C3E8A110A124C278A110A1231
:10128000712F3D03230203190800B1002030B00084
:101290008A110A122F2709308A00B10B48298A11B6
:1012A0000A12712F831203132B304802031D5C298D
:1012B00083120313060A67292D304802031D64298F
:1012C00083120313060367298312031348080F3997
:1012D00083120313B10083120313F03086058312C7
:1012E00003133108831203138604831203130800C7
:1012F00083120313C80883120313031D81290612E6
:101300000800061608000C308A002930480203182D
:10131000262C4808A300053049020318262C49084A
:10132000A200221C97290830A3000230A200080066
:10133000831203130730D10551088313E03E840064
:1013400050088000D10DD10DD10D5108403E8A11B9
:101350000A124C2783134F3084000830B200000873
:10136000B0008A110A122F2709308A008403B20BB9
:10137000AF298A110A12712F080083120313543007
:10138000E0003A30E1006D086E1F803A6E13E20013
:101390000330EB008A110A126F2E4808AB0049088F
:1013A000A700A71927124A08AA004B08A9004C0851
:1013B000A800080083120313060883120313AD006C
:1013C0008A150A1264268316031706308C19153005
:1013D00083120313E0000130EB008A110A126F2E12
:1013E00003104E084D074C074B074A0749074802B0
:1013F000031D262C0630B10083134E3084000130CB
:10140000B90000088A110A128625B90A84030A3035
:101410008A00B10B012A08000030B90000308A119F
:101420000A1286258A110A12002883120313261035
:1014300048182614A510C818A514241048192414F7
:101440002613A412C819A4162611C81A2615A61107
:10145000481BA61524132513481E0800241725171A
:10146000080083120313C80126184814A518C814CD
:1014700024184815A41AC815241B48162619C8167E
:10148000A6194817831203134B30E0004D30E100DA
:101490003A30E2000330EB008A110A126F26013065
:1014A000C1008A150A120028831203134B30E00092
:1014B0005030E1003A30E2000330EB008A110A12AA
:1014C0006F2683134808A83E84000008C800013036
:1014D000C1008A150A120028831203134B30E00062
:1014E0004530E1003A30E2000330EB008A110A1285
:1014F0006F264030B1007F30BB00BA01A6168A11BA
:101500000A12AB25B200AA308A110A12F625013060
:10151000B0008A110A12AB25AA3C031DB0010A30A3
:101520008A003A1E9B2A3A128A110A12AB25AA3C5B
:101530000319B0013A1632088A110A12F62530084A
:101540002618303EE0000130EB008A110A126F26A7
:101550000A308A00BA0AB10B7F2A261CB62A3B3011
:10156000E0000130EB008A110A126F268A110A127C
:10157000EA268A110A121E29A61048080319A0019A
:10158000A0080319A0002002031908004808FF3C26
:1015900003190800A6140800831203135430E00056
:1015A0004B30E1003A30E2000330EB008A110A12BE
:1015B0006F262808CC002908CB002A08CA00270873
:1015C000C9002B08C8000530C1008A150A1200287E
:1015D000CA034A081F39203EB90049088A110A1275
:1015E00086254A081F39503EB90048088A110A1258
:1015F0008625831203130800831203135430E0007E
:101600004330E1003A30E2000330EB00C803480801
:101610001F39B300203EB9008A110A1279258312BE
:101620000313E3000A308A002618262B3308503EA5
:10163000B9008A110A12792583120313E4000A30D3
:101640008A000530EB008A110A126F2E2C30E4005C
:101650003308503EB9008A110A1279258312031308
:10166000E5000A308A003B30E6000730EB008A11C3
:101670000A126F2E4A080739A03E8400831300081F
:10168000C808031D452B49084B2B481C482B49040F
:10169000C81C4B2B4906800083120313080048081E
:1016A00007398313B03E84008316031300088312A6
:1016B0000313C800831203135030E0004930E100E7
:1016C0003A30E2000330EB008A110A126F26013033
:1016D000C1008A150A120028831203132612481922
:1016E00026164808033983120313AC008A150A1220
:1016F000642E83120313480883120313E0000130A1
:10170000EB008A110A126F2E831203134908BA00E4
:101710004808BB008A110A12AB2583120313E000AC
:10172000C8000B308A0026189A2B0130EB008A1172
:101730000A126F2E831203134530E0003A30E100A5
:101740000230EB008A110A126F260130C1008A159F
:101750000A120028831203134A08BA004908BB0082
:1017600048088A110A12F625E0000130EB008A11C0
:101770000A126F2E83120313E0010310003050078A
:101780004F074E074D074C074B074A0749074802CA
:101790000319CD2B1530E000DF2B0830B100831387
:1017A0005030840000088A110A12F625E007BB0AAF
:1017B0000319BA0A84030B308A00B10BD22B013013
:1017C000EB008A110A126F2EFE303602031DEB2B3E
:1017D0004808B60008004808B600360DFE39BB00C0
:1017E0000130BA00FE30B6002608F900A6108A11B2
:1017F0000A12AB25B1008A110A12DB25BB003108A1
:10180000BA008A110A12AB25B1000C308A003108E7
:101810000319162C8A110A1216228A110A12DB25C4
:1018200083120313B1000C308A00072C7908A6003C
:10183000FE3036020319B60A080048080739A1002D
:1018400008004808B7004908D700080005308A1189
:101850000A12742E0C308A0083120313EE1808004B
:101860006E110430F400F501B20183162008F0393E
:10187000E8000730A00083162008A01D0B30201DB3
:101880000D30A01C0E30201C0730A0006808A004FA
:1018900083128A110A12E4210C308A008312031386
:1018A0008313B0308400B101800C03185B2C310825
:1018B000B200B20A5F2CB10AB11D542C692C740815
:1018C000B3000830B207B30B622CB2023208F50045
:1018D0005B2CF40B3B2C7508B0000319982C6E168A
:1018E0006E15982C0C308A006E190800EE106E12DE
:1018F0007208B20003190800B001B1018313B130BE
:1019000084000830B300800CB10A031C8E2CB30B8A
:10191000832CB2030319972C840A812C2B083102E3
:10192000031D942C6E16872C3108B000872CEE1402
:10193000B008031DB62C271EA62C7208B200831314
:10194000A03E840080018403B20BA22C83120313F7
:101950006E12EE12EE13EE106E11B201EC01EE1DDE
:10196000E12CEE11271DE12C6E17E12CEE1EBC2C94
:1019700030086C020319E22CEE16EE132808F10071
:101980003008EC00E12CA71EC92C8312031305308C
:10199000B400271EE12C7208B2008313A03E84001D
:1019A00080018403B20BD02C8313A1308400300853
:1019B000B1000314800D031CDF2C840A800DB10BD1
:1019C000DA2C0800F10BE12CEE1BFB2CA718EE170C
:1019D0002908F100EE1D6E17EE156C036E1A303EED
:1019E000203EB9008A110A127925ED000C308A00D8
:1019F0006E1BC32CE12C6E172A08F100C32C8B013F
:101A00008A118C0185018601051683160313C030E7
:101A1000860009308500831603130E309F0083165D
:101A200003178C0107308100831603138C018C1679
:101A3000831203138B010B178B17101490101016C1
:101A400090160A309B000A309C00831203138130E9
:101A50009F00831603130E309F008312031394120A
:101A60008701071705168316031398308700831222
:101A700003132830940083160313803094008316D8
:101A80000313193093008312031308002030B100B0
:101A90008313A03084008001840AB10B4B2D1030D9
:101AA000B1008313203084001030B90039088A1146
:101AB0000A1279258000B90A840A0D308A00B10B18
:101AC000562D2D0883120313860083120313013051
:101AD000BC00BD008A110A1271270D308A008312E2
:101AE00003130330B400A008031DA614FF30B50093
:101AF000B600B700D701EC0138308100E901E801F8
:101B0000EB01EA01EE01BF01C301C401C501C60139
:101B1000C7010330C200BA01BB01A6168A110A121E
:101B2000AB25B100AA308A110A12F6251030BA008E
:101B30008A110A12AB25B00055308A110A12F62517
:101B4000BA018A110A12AB25553C0319A6123108B5
:101B50008A110A12F6252030BA0030088A110A12BA
:101B6000F62508000830B1008313A83084008312E2
:101B70000313051600000000851200000512053051
:101B80008A00003009250F3980000D308A00840A50
:101B9000B10BBF2D831603130830A8008312031363
:101BA0000830F300AF308400000A0F39031DDB2D2D
:101BB0008403F30BD42DF2017208A93E8400013096
:101BC0000002031DE82DF20A04307202031DDC2D11
:101BD00083120313F2080319A412A71D0800A41608
:101BE000080083160313243098000E308A000B136C
:101BF000831203132C080339092683160313990053
:101C000083120313903098008312031387120B176B
:101C100008008207813440342034143400308A11A3
:101C20000A127925013C031908000430A20014307F
:101C3000A3008A150A12E7200A308A110A127426B4
:101C4000831203130130AC00A001A1012730AD00C5
:101C50000A30A8006430A9002830AA00A601261482
:101C60002615A701A714A71627162708AB01A4015C
:101C7000A414A514A416241725172408A5002030A1
:101C8000B1003F30B9003108603E8A110A12862542
:101C90000E308A0083120313B903B10B432E203098
:101CA000B1006F30B9003108403E8A110A12862512
:101CB0000E308A0083120313B903B10B532EB901FE
:101CC00001308A110A1286251030B1008313831265
:101CD0000313203084001030B90000088A110A1262
:101CE0008625B90A840A0E308A00B10B6D2E0800D1
:101CF00083120313BE013E14BE143E15BE153E12E0
:101D0000831603130908F839890008080030880091
:101D100083128A110A12DE268A110A12DE268A111D
:101D20000A12DE260E308A00890133308800091439
:101D30008616000000000910861200008A110A129F
:101D4000EA260914861600000000091086120630E3
:101D50008A005430ED260E308A00091486160000E1
:101D60000000091086128A110A12EA2630308A1100
:101D70000A124C278A110A12EA263E163C303E1DF2
:101D80008011BE1D00118A110A124C27BA01BB0135
:101D900040308A110A124C278A110A12AB25B00072
:101DA0008A110A122F270E308A00BB0A3B1FCC2E45
:101DB0000830B1008313E03084008A110A12AB2589
:101DC0008000840A0E308A00BB0AB10BDD2E083079
:101DD0008A110A124C2701308A110A124C278A11E3
:101DE0000A12EA260F303E1A0C308A110A124C27CA
:101DF00006308A110A124C273E1E08003E120E3091
:101E00008A00BE2E8312031326190B2FC8018A15D0
:101E10000A12E42308008A11013074262C30B00025
:101E2000F426043074264830840023088A110A12EC
:101E3000A3274808B000F4260F308A006B18252F1E
:101E40004908B0008A110A12F4267830B0008A11CD
:101E50000A12F4262208303EB0008A110A12F42633
:101E60000F308A000830230203196A2F0130BD00A9
:101E70000230BC008A110A1271278A110230261A18
:101E800003307426831203132C08063E74260F3089
:101E90008A00A61C6A2F4830840020088A110A1282
:101EA000A3270B3074264808B000F4260F308A00B0
:101EB000EB0B5B2F6A2F4908B0008A110A12F42637
:101EC0000F308A00EB0B652F6A2F4A08B0008A1189
:081ED0000A12F426EB010800E0
:02400E00321D61
:00000001FF
